 BulkUsb

 Timestamp is 3fd02d19 (Fri Dec 05 15:00:41 2003)

 Preferred load address is 00010000

 Start         Length     Name                   Class
 0001:00000000 0000167eH .text                   CODE
 0002:00000000 00000090H .idata$5                DATA
 0002:00000090 00000068H .rdata                  DATA
 0003:00000000 0000003cH .idata$2                CODE
 0003:0000003c 00000014H .idata$3                CODE
 0003:00000050 00000090H .idata$4                CODE
 0003:000000e0 000002eaH .idata$6                CODE
 0004:00000000 00000058H .rsrc$01                DATA
 0004:00000060 00000350H .rsrc$02                DATA

  Address         Publics by Value              Rva+Base     Lib:Object

 0001:00000000       _DriverEntry@8             000102a0 f   bulkusb.obj
 0001:0000005c       _BulkUsb_ProcessSysControlIrp@8 000102fc f   bulkusb.obj
 0001:000000ae       _BulkUsb_Unload@4          0001034e f   bulkusb.obj
 0001:000000b2       _BulkUsb_SymbolicLink@8    00010352 f   bulkusb.obj
 0001:000000da       _BulkUsb_CreateDeviceObject@12 0001037a f   bulkusb.obj
 0001:000001a8       _BulkUsb_CallUSBD@8        00010448 f   bulkusb.obj
 0001:00000216       _BulkUsb_ConfigureDevice@4 000104b6 f   bulkusb.obj
 0001:000002ce       _BulkUsb_SelectInterface@8 0001056e f   bulkusb.obj
 0001:000003fa       _BulkUsb_ResetPipe@8       0001069a f   bulkusb.obj
 0001:00000448       _BulkUsb_DecrementIoCount@4 000106e8 f   bulkusb.obj
 0001:000004b2       _BulkUsb_IncrementIoCount@4 00010752 f   bulkusb.obj
 0001:000004e8       _BulkUsb_ProcessPnPIrp@8   00010788 f   bulkpnp.obj
 0001:0000075e       _BulkUsb_PnPAddDevice@8    000109fe f   bulkpnp.obj
 0001:000007fc       _BulkUsb_StartDevice@4     00010a9c f   bulkpnp.obj
 0001:000008b6       _BulkUsb_RemoveDevice@4    00010b56 f   bulkpnp.obj
 0001:0000092a       _BulkUsb_StopDevice@4      00010bca f   bulkpnp.obj
 0001:00000988       _BulkUsb_IrpCompletionRoutine@12 00010c28 f   bulkpnp.obj
 0001:0000099e       _BulkUsb_ProcessPowerIrp@8 00010c3e f   bulkpwr.obj
 0001:00000b7a       _BulkUsb_PoRequestCompletion@20 00010e1a f   bulkpwr.obj
 0001:00000bce       _BulkUsb_PowerIrp_Complete@12 00010e6e f   bulkpwr.obj
 0001:00000bfe       _BulkUsb_SelfSuspendOrActivate@8 00010e9e f   bulkpwr.obj
 0001:00000c04       _BulkUsb_SetDevicePowerState@8 00010ea4 f   bulkpwr.obj
 0001:00000c32       _BulkUsb_QueryCapabilities@8 00010ed2 f   bulkpwr.obj
 0001:00000cc2       _BulkUsb_ProcessIOCTL@8    00010f62 f   ioctlblk.obj
 0001:00000d96       _BulkUsb_ResetDevice@4     00011036 f   ioctlblk.obj
 0001:00000dc2       _BulkUsb_GetPortStatus@8   00011062 f   ioctlblk.obj
 0001:00000e34       _BulkUsb_ResetParentPort@4 000110d4 f   ioctlblk.obj
 0001:00000e9a       _BulkUsb_SingleUrbReadWrite@12 0001113a f   ocrwblk.obj
 0001:00000f28       _BulkUsb_StagedReadWrite@12 000111c8 f   ocrwblk.obj
 0001:000011de       _BulkUsb_BuildAsyncRequest@16 0001147e f   ocrwblk.obj
 0001:00001248       _BulkUsb_AsyncReadWrite_Complete@12 000114e8 f   ocrwblk.obj
 0001:0000131c       _BulkUsb_SimpleReadWrite_Complete@12 000115bc f   ocrwblk.obj
 0001:0000136a       _BulkUsb_Read@8            0001160a f   ocrwblk.obj
 0001:0000137c       _BulkUsb_Write@8           0001161c f   ocrwblk.obj
 0001:0000138e       _BulkUsb_PipeWithName@8    0001162e f   ocrwblk.obj
 0001:00001410       _BulkUsb_Close@8           000116b0 f   ocrwblk.obj
 0001:00001474       _BulkUsb_Create@8          00011714 f   ocrwblk.obj
 0001:00001544       _BulkUsb_CancelPendingIo@4 000117e4 f   ocrwblk.obj
 0001:000015a8       _BulkUsb_AbortPipes@4      00011848 f   ocrwblk.obj
 0001:00001650       _BulkUsb_CanAcceptIoRequests@4 000118f0 f   ocrwblk.obj
 0002:00000000       __imp_@KfAcquireSpinLock@4 00011920     wdm:HAL.DLL
 0002:00000004       __imp_@KfReleaseSpinLock@8 00011924     wdm:HAL.DLL
 0002:00000008       \177HAL_NULL_THUNK_DATA    00011928     wdm:HAL.DLL
 0002:0000000c       __imp__KeInitializeSpinLock@4 0001192c     wdm:NTOSKRNL.EXE
 0002:00000010       __imp__KeInitializeEvent@12 00011930     wdm:NTOSKRNL.EXE
 0002:00000014       __imp__RtlFreeUnicodeString@4 00011934     wdm:NTOSKRNL.EXE
 0002:00000018       __imp__IoCreateDevice@28   00011938     wdm:NTOSKRNL.EXE
 0002:0000001c       __imp__IoSetDeviceInterfaceState@8 0001193c     wdm:NTOSKRNL.EXE
 0002:00000020       __imp__IoRegisterDeviceInterface@16 00011940     wdm:NTOSKRNL.EXE
 0002:00000024       __imp__ExFreePool@4        00011944     wdm:NTOSKRNL.EXE
 0002:00000028       __imp__ExAllocatePoolWithTag@12 00011948     wdm:NTOSKRNL.EXE
 0002:0000002c       __imp__IoBuildDeviceIoControlRequest@36 0001194c     wdm:NTOSKRNL.EXE
 0002:00000030       __imp__KeSetEvent@12       00011950     wdm:NTOSKRNL.EXE
 0002:00000034       __imp_@InterlockedDecrement@4 00011954     wdm:NTOSKRNL.EXE
 0002:00000038       __imp__KeWaitForSingleObject@20 00011958     wdm:NTOSKRNL.EXE
 0002:0000003c       __imp_@InterlockedIncrement@4 0001195c     wdm:NTOSKRNL.EXE
 0002:00000040       __imp_@IofCompleteRequest@8 00011960     wdm:NTOSKRNL.EXE
 0002:00000044       __imp__IoDeleteDevice@4    00011964     wdm:NTOSKRNL.EXE
 0002:00000048       __imp_@IofCallDriver@8     00011968     wdm:NTOSKRNL.EXE
 0002:0000004c       __imp__IoAttachDeviceToDeviceStack@8 0001196c     wdm:NTOSKRNL.EXE
 0002:00000050       __imp__RtlInitUnicodeString@8 00011970     wdm:NTOSKRNL.EXE
 0002:00000054       __imp__PoRequestPowerIrp@24 00011974     wdm:NTOSKRNL.EXE
 0002:00000058       __imp__PoCallDriver@8      00011978     wdm:NTOSKRNL.EXE
 0002:0000005c       __imp__PoStartNextPowerIrp@4 0001197c     wdm:NTOSKRNL.EXE
 0002:00000060       __imp__IoFreeIrp@4         00011980     wdm:NTOSKRNL.EXE
 0002:00000064       __imp__IoAllocateIrp@8     00011984     wdm:NTOSKRNL.EXE
 0002:00000068       __imp__IoBuildPartialMdl@16 00011988     wdm:NTOSKRNL.EXE
 0002:0000006c       __imp__IoAllocateMdl@20    0001198c     wdm:NTOSKRNL.EXE
 0002:00000070       __imp__IoFreeMdl@4         00011990     wdm:NTOSKRNL.EXE
 0002:00000074       __imp__IoCancelIrp@4       00011994     wdm:NTOSKRNL.EXE
 0002:00000078       __imp__IoDetachDevice@4    00011998     wdm:NTOSKRNL.EXE
 0002:0000007c       \177NTOSKRNL_NULL_THUNK_DATA 0001199c     wdm:NTOSKRNL.EXE
 0002:00000080       __imp__USBD_CreateConfigurationRequest@8 000119a0     usbd:USBD.SYS
 0002:00000084       __imp__USBD_GetUSBDIVersion@4 000119a4     usbd:USBD.SYS
 0002:00000088       __imp__USBD_ParseConfigurationDescriptorEx@28 000119a8     usbd:USBD.SYS
 0002:0000008c       \177USBD_NULL_THUNK_DATA   000119ac     usbd:USBD.SYS
 0002:000000e8       _GUID_CLASS_ZHONGQING_VIDEO_DEV 00011a08     bulkusb.obj
 0003:00000000       __IMPORT_DESCRIPTOR_NTOSKRNL 00011a20     wdm:NTOSKRNL.EXE
 0003:00000014       __IMPORT_DESCRIPTOR_HAL    00011a34     wdm:HAL.DLL
 0003:00000028       __IMPORT_DESCRIPTOR_USBD   00011a48     usbd:USBD.SYS
 0003:0000003c       __NULL_IMPORT_DESCRIPTOR   00011a5c     wdm:NTOSKRNL.EXE

 entry point at        0001:00000000

 Static symbols

